:020000040800F2
:10000000E855002081020008AB350008AD3100083A
:10001000A9350008C50300088D4100080000000054
:10002000000000000000000000000000A101000826
:10003000C107000800000000FD010008033C0008A3
:100040009B0200089B0200089B0200080D38000874
:100050009B0200089B0200089B0200089B0200080C
:100060009B0200089B0200089B0200089B020008FC
:100070009B0200089B0200089B0200089B020008EC
:10008000A9070008B50700089B020008E103000863
:10009000C90300089B020008D50300089B02000862
:1000A0009B0200089B0200089B0200089B020008BC
:1000B0009B02000800000000000000009B020008F6
:1000C0009B0200089B0200089B0200089B0200089C
:1000D0009B0200089B020008814100089B02000867
:1000E0009B0200089B0200080000000000000000C6
:1000F0000000000000000000000000000000000000
:10010000000000009B020008000000009B020008A5
:100110000000000000000000BD3C00089B02000839
:100120009B0200089B0200089B0200089B0200083B
:100130009B0200080000000000000000000000001A
:100140009B0200089B0200089B02000800000000C0
:100150009B0200089B0200089B0200089B0200080B
:100160009B0200089B0200089B02000800000000A0
:100170009B0200089B020008000000000000000035
:100180009B0200089B0200089B020008DFF80CD0CD
:1001900000F006F90048004769470008E8550020CC
:1001A0002C4B1968086800F05AB880F30988BFF32F
:1001B0006F8F4FF0000080F311887047000000003F
:1001C00008480068006880F308884FF0000080F35A
:1001D000148862B661B6BFF34F8FBFF36F8F00DF35
:1001E00000BF00BF08ED00E0DFF80C00016841F43B
:1001F00070010160704700BF88ED00E0EFF30980F7
:10020000BFF36F8F134B1A681EF0100F08BF20ED5D
:10021000108A20E9F04F106009B44FF0500080F3CD
:100220001188BFF34F8FBFF36F8F05F0A7FA4FF020
:10023000000080F3118809BC1968086800F014B840
:100240001EF0100F08BF00F014B880F30988BFF348
:100250006F8F704768000020EFF30580704730C84B
:10026000B0E8C04FFFF7A1BF30C8B0E8C04FFFF7FC
:10027000E7BFB0EC088AB0EC08CAFFF7E6BF0000A1
:100280000648804706480047FEE7FEE7FEE7FEE730
:10029000FEE7FEE7FEE7FEE7FEE7FEE7AD3C00080F
:1002A0008D0100082DE9F05F0546002092469B462F
:1002B00088460646814640241BE02846414647467C
:1002C000224600F05DF853465A46C01A914110D3B9
:1002D00011461846224600F044F82D1A67EB010833
:1002E0004F4622460120002100F03BF817EB0009A1
:1002F0004E41201EA4F10104DFDC484631462A4667
:10030000434600F000B830BCBDE8C09F40EA01039E
:100310009B0703D009E008C9121F08C0042AFAD2BB
:1003200003E011F8013B00F8013B521EF9D270477F
:10033000D2B201E000F8012B491EFBD27047002227
:10034000F6E710B513460A4604461946FFF7F0FFD4
:10035000204610BD421C10F8011B0029FBD1801A59
:100360007047202A04DB203A00FA02F1002070478F
:100370009140C2F1200320FA03F3194390407047E3
:10038000202A04DB203A21FA02F00021704721FAEA
:1003900002F3D040C2F12002914008431946704751
:1003A000064C074D06E0E06840F0010394E80700C2
:1003B00098471034AC42F6D3FFF7ECFE28640008EF
:1003C00048640008FEE70000014800F043BD00005B
:1003D00064010020014800F03DBD000064010020E0
:1003E000014800F037BD00006401002030B58BB03B
:1003F00000200124CDE90604059004908020042506
:10040000CDE900054FF6FF7008940290039069460D
:100410000F4800F031FC40B988200594CDE9000573
:1004200069460B4800F028FC20B100F007FA0120D3
:100430000BB030BD064800F00EFE0028F8D004488E
:1004400000F092FC014603A003F0CAFEEDE70000B5
:100450006401002043414E20496E697469616C69F2
:100460007A6174696F6E204572726F723A20256CE2
:10047000640A000030B587B01205DDE90A4542EA9A
:10048000033242EA042242EA051242F0805201920B
:10049000042202920022CDE90321024606AB6946FE
:1004A000074800F08AFB010007D006A003F098FE81
:1004B0000348416A10A003F093FE07B030BD00006E
:1004C0006401002048414C5F43414E5F41646454E5
:1004D000784D657373616765206661696C6564203A
:1004E0002C207265745F7374617475733A3078256B
:1004F00078200D0A000000006863616E2D3E457291
:10050000726F72436F64653A2030782578200D0A47
:1005100000000000F0B589B00024DDE90E5600941B
:100520000194178800063F0A8DF8007017788DF83F
:10053000017092788DF80220000940EA033005F03E
:100540000F0240EA022006F00F0240EA0210039078
:10055000042004908DF803400194CDE9054108ABD7
:100560006A4602A9074800F028FB010007D006A050
:1005700003F036FE0348416A10A003F031FE09B0D3
:10058000F0BD00006401002048414C5F43414E5FD4
:1005900041646454784D6573736167652066616971
:1005A0006C6564202C207265745F7374617475735C
:1005B0003A30782578200D0A000000006863616EEB
:1005C0002D3E4572726F72436F64653A2030782514
:1005D00078200D0A00000000F0B587B00D460746F0
:1005E000DDE90C101206120942EA033201F00F0194
:1005F00042EA012100F00F0041EA001001900420BE
:1006000002900020CDE9030506AB3A46694613483F
:1006100000F0D3FA20B112A003F0E2FD07B0F0BD64
:1006200005EB450004F0D6F8064600240AE000BFBA
:1006300004EB440037F81420304410A103F0E0FD2F
:10064000641CE4B2AC42F3D332460EA0019903F02D
:10065000C7FD304604F060F8E0E7000064010020C8
:1006600043414E206D6573736167652073656E64E9
:10067000206661696C65640A00000000253032580C
:100680002000000043414E206D6573736167652053
:1006900073656E743A2049443D3078253038582CC3
:1006A00020446174613D25730A0000000A2004F0B3
:1006B000C7F8FBE770B586B014216846FFF73FFE28
:1006C0002C4C54F84C0F40F001002060206800F0E2
:1006D00001000590206840F002002060206800F0D2
:1006E00002000590606C40F400406064E06840F4F3
:1006F0000030E060E0684FF0904500F40030059075
:1007000003200190002002904FF6FF700090694690
:10071000284601F037F847F6FF70174E00906946FB
:10072000304601F02FF801224FF4F051284601F035
:1007300019F9012248F20101304601F013F90022B3
:100740001021304601F00EF9206820F001002060F1
:10075000206820F002002060E06820F40030E060B3
:10076000E06820F40010E060E06820F00070E060D5
:1007700006B070BD001002400004004800EE100AF0
:100780009FED071AF8EE400A80EE810AF3EE090A9F
:1007900020EE200ADFED030A20EE200A7047000059
:1007A00000FC7F460000C842014800F04ABE00003D
:1007B00034020020014800F044BE00007C0200200A
:1007C0007047000010B50446064801F03BFF0422C4
:1007D0002146044801F07CFF2146BDE8104002A0FC
:1007E00003F0FEBC8C0100205254432057616B651E
:1007F00075702054696D65722073657420666F7220
:1008000020256420730A000010B507A003F0E8FC5F
:10081000FFF750FF08488078FFF7D4FFBDE810408D
:10082000012001F09DB90000456E746572696E6724
:100830002053746F70320A000600002072B6FEE783
:10084000144A117F1448012901D003290FD10368EC
:1008500023F400730360036843F4006303600368D8
:1008600023F400630360036843F400730360022908
:1008700001D003290BD1016841F480510160016866
:1008800021F480510160016841F480610160002021
:10089000107770474400002000200240C10705483F
:1008A00003D0416941F004014161416941F4803163
:1008B000416170470020024008494A69C0B222F4F1
:1008C0007E7242EAC0004861486940F00200486117
:1008D000486940F4803048617047000000200240C1
:1008E000054910B54C6944F001044C610260BFF346
:1008F0006F8F436010BD000000200240094A10B510
:100900005469402344F480245461EFF3108272B69A
:1009100010C910C05B1E13F0FF03F9D182F31088D9
:1009200010BD00000020024070B5054601F020F81F
:100930000646134C08E0681C06D001F019F8801B2D
:10094000A84201D3032070BD2069C003F3D42069FD
:100950000C4908400CD00C494A6802434A60810F98
:1009600001D0A169A161810000D02061012070BD8A
:100970002069C00701D001202061002070BD000067
:1009800000200240FAC302004400002070B586B087
:100990000C00054628D01548854225D80026049627
:1009A00000F0DCFE1248816941F0404181614CF267
:1009B000FA3101612846009600F01CF801902846A3
:1009C00000F026F8029005EB8400401E00F020F8AD
:1009D0000299401A401C039004A9684600F0EEFDFD
:1009E000002801D000F05AFE06B070BD00000408D7
:1009F000002002400449096804494FF001000968D9
:100A0000CA431204120C704700000140E075FF1F3A
:100A10000E4910B509684FF48024CB431A04120C18
:100A20000AD00A045FEA921202F10062824205D9FA
:100A3000A0F10060C00A10BD2246F5E71A04120CAE
:100A400001D009048C09001BF2E70000E075FF1FCC
:100A5000064B10B5984207D8002303E010F8014B6D
:100A6000CC545B1C9342F9D310BD00000000040875
:100A70002DE9F04117460D46044600F06FFE0F4881
:100A8000844216D2002609E0D5E900232146002041
:100A900000F00EFE68B908340835761CB6EB570F27
:100AA000F2D3F80705D06368214600202A6800F0D9
:100AB000FFFDBDE8F04100F0F1BD000000000408BA
:100AC0002DE9F04FE5B0994614460E0083460CD050
:100AD000A1074FEA940000D0401C00271FFA80FABB
:100AE0008DF800703D46E8460CE0012065B000F04E
:100AF0004FB86846FFF72EFC4044725D17A103F023
:100B00007FFB6D1CA542F4D3694616A003F068FB79
:100B100001215846FFF73AFF524631465846FFF743
:100B2000A7FF224649465846FFF792FF8DF8C87046
:100B3000002532AE09E032A8FFF70CFC304419F86A
:100B4000052006A103F05CFB6D1CA542F3D332A97E
:100B500009A003F045FB0020C8E70000253032580B
:100B600020000000466C6173685F577269746533DA
:100B7000323A2025730D0A00466C6173685F526536
:100B8000616442797465733A2025730D0A00000090
:100B900030BCBDE8C08F90F82020012A07D0022A7F
:100BA00005D0416A41F4802141620120704700680C
:100BB00042690A43426100207047F0B590F8205026
:100BC0000468A468012D05D0022D03D0416A41F4C8
:100BD00080214DE014F0406F01D1E50045D5C4F30C
:100BE00001640125A5401D608D684FF4C0739DB15F
:100BF000CE6835434E6845EAC605066803EB041720
:100C0000F5514FF4C275076805EB04150E697E5166
:100C1000097D012905D009E00E88CD6845EA4655D1
:100C2000EBE701684E5946F480764E511179D2F8BF
:100C300005504FF4C67641EA0521056806EB041617
:100C4000A9511178D2F801204FF4C47541EA02216C
:100C5000026805EB04155151006803EB041142587A
:100C600042F0010242500020F0BD416A41F40011FF
:100C700041620120F0BD000010B590F820300268FC
:100C8000012B07D0022B05D0416A41F4802141623B
:100C9000012010BDD2F8000240F00100C2F80002AD
:100CA000087D00F01F0301209840D2F81C328343D6
:100CB000C2F81C32CB69B3B9D2F80C328343C2F804
:100CC0000C328C894B6864F31F434C6902EBC404FB
:100CD000C4F840320C890B6864F31F434C6902EB83
:100CE000C404C4F84432CB69012B16D1D2F80C32BB
:100CF0000343C2F80C320C884B6864F31F434C6901
:100D000002EBC404C4F840320C89CB6864F31F437F
:100D10004C6902EBC404C4F844328B69002BD2F84E
:100D200004320FD053EA0003C2F804320B69002BDF
:100D3000D2F8143208D00343C2F81432096A0129E8
:100D400004D008E08343EFE78343F5E7D2F81C12B1
:100D50000143C2F81C12D2F8000220F00100C2F8D0
:100D60000002002010BD7047406A704730B590F80F
:100D70002040012C05D0022C03D0416A41F480218F
:100D80005DE00468002955D02469A40754D04FF4CD
:100D9000D874056804EB01142D5915F0040595600D
:100DA00005682D594ED0ED08556005682C5904F0A2
:100DB0000204D4604FF4DA74056804EB01142D5971
:100DC00005F00F05156105682D59C5F307259561D7
:100DD00005682C59240C54614FF4DC72046802EB52
:100DE0000112A4581C700468A458240A5C7004689A
:100DF000A458240C9C700468A258120EDA704FF4A8
:100E0000DE72046802EB0112A4581C710468A45835
:100E1000240A5C710468A458240C9C710468A258CC
:100E2000120EDA71006881B1016941F0200101619F
:100E3000002030BDE468A8E7416A41F40011416236
:100E4000012030BD6D0D1560AFE7C16841F0200194
:100E5000C160EDE72DE9F05F0546006800244669B2
:100E6000D0F804908768D0F80CB0D0F810A0D0F873
:100E70001880F10748D0F90714D001218160B80724
:100E800003D5284600F08BFA0CE0780702D54FF422
:100E9000006407E0380702D54FF4805402E028468A
:100EA00000F07CFAF80516D529684FF48070886048
:100EB000B80503D5284600F074FA0CE0780502D591
:100EC00044F4005407E0380502D544F4804402E0BD
:100ED000284600F065FAF80316D529684FF48030EB
:100EE0008860B80303D5284600F05DFA0CE078036B
:100EF00002D544F4004407E0380302D544F48034BA
:100F000002E0284600F04EFA300707D55FEACB60D2
:100F100004D52968102044F40074C86070074FF0AD
:100F2000080707D55FEA0B7004D52868C760284614
:100F300000F068F9B00706D52868C068800702D0BD
:100F4000284600F061F9700607D55FEACA6004D54B
:100F50002968102044F480640861B00607D55FEA70
:100F60000A7004D528680761284600F0E7F9F00602
:100F700006D528680069800702D0284600F0DFF90E
:100F8000B00308D55FEAC96005D52968102048601C
:100F9000284600F0D5F9F00307D55FEA097004D5BB
:100FA00028684760284600F0FFF9300446D55FEA1C
:100FB000497040D5F00504D55FEAC87001D044F00F
:100FC0000104B00504D55FEA887001D544F002043D
:100FD000700504D55FEA487001D544F0040430057B
:100FE00029D518F0700F26D008F07000402815D0D1
:100FF00006DC102809D020280AD0302816D10AE0B3
:1010000050280ED0602811D10EE044F008040DE005
:1010100044F010040AE044F0200407E044F04004E7
:1010200004E044F0800401E044F48074286881699D
:1010300021F070018161296804204860002C05D0EE
:10104000686A204368622846FFF78DFE00F000B80A
:1010500030BCBDE8C09F70B5040003D094F82000F8
:1010600010B104E0012070BD204600F081F8206836
:10107000016841F00101016000F07AFC0546052697
:1010800004E000F075FC401B0A2811D82068406875
:10109000C007F6D02068016821F00201016000F06D
:1010A00067FC05460BE000F063FC401B0A2806D9EC
:1010B000606A40F40030606284F82060D2E7206803
:1010C00040688007EFD4207E0128206801683DD069
:1010D00021F080010160607E01282068016838D01D
:1010E00021F040010160A07E01282068016833D012
:1010F00021F020010160E07E0128206801682ED0E7
:1011000041F010010160207F01282068016829D08A
:1011100021F008010160607F01282068016824D067
:1011200021F004010160D4E902010843D4E904126A
:10113000114308436168491E08432168C8610020C3
:101140006062012084F82000002070BD41F0800121
:10115000C0E741F04001C5E741F02001CAE721F0B6
:101160001001CFE741F00801D4E741F00401D9E7CD
:1011700010B586B0044614216846FFF7E0F81F4911
:101180002068884237D11E48816D41F00071816529
:10119000816D01F000710591C16C41F00101C164E4
:1011A000C06C694600F0010005904FF4C0500090FB
:1011B0000220019000200290032003900920049057
:1011C000C00600F0DFFA00220521132000F062FCC7
:1011D000132000F051FC00220521142000F05AFCDD
:1011E000142000F049FC00220521162000F052FCDA
:1011F000162000F041FC06B010BD00000064004065
:10120000001002407047000030B58BB002AB04AA5A
:1012100000213248FFF7AAFD40B13048FFF7A4FD96
:1012200001462FA002F0DCFF0BB030BD0598FF2473
:10123000354DB0F5801F03D0B0F5881F24D026E0CF
:101240000698042823D131A0059902F0C9FF9DF822
:10125000090090B19DF80810FF2902D02A78914228
:10126000E2D1288002F010FC00940194FF232A8828
:1012700001212548FFF7B0F9D6E7234AFF23921C46
:1012800000940021019424E00698042803D025A0AE
:1012900002F0A6FFC8E71DA0059902F0A1FF9DF886
:1012A0000C0018B99DF80D000028E6D09DF80E102E
:1012B0000029E2D0144ABDF80C00921C40BA1080FC
:1012C000917002F019FC104AFF23921C0094032134
:1012D00001942888FFF71EF9A6E7000064010020AA
:1012E00043414E2072656365697665206661696C6D
:1012F0006564214572726F7220636F64653A2030B5
:10130000782530386C580A000400002043414E49CB
:10131000442072656365697665643A2030782530CB
:1013200038580A0043414E4944206D69736D617419
:1013300063686564EFBC815C6E00000070477047B5
:101340007047000070B5044690F82000012804D0D2
:10135000606A40F40020606218E0022084F82000F7
:101360002068016821F00101016000F001FB0546E1
:101370000EE000BF00F0FCFA401B0A2808D9606AA2
:1013800040F400306062052084F82000012070BD28
:1013900020684068C007EDD1606270BD704770473B
:1013A0007047704770477047704710B590F8251028
:1013B0000022022905D00421C16380F824200120E5
:1013C00010BD01680B6823F00E030B6001680B6809
:1013D00023F001030B6090F84410046C01F01C032F
:1013E000012101FA03F3636080F8251080F82420BE
:1013F000104610BD10B590F825100024022903D026
:101400000421C16301241AE001680A6822F00E0277
:101410000A6001680A6822F001020A6090F844102C
:10142000036C01F01C02012101FA02F25A6080F8FB
:101430002510002180F82410816B01B188472046D7
:1014400010BDF0B4016C0C6801680D6890F8442080
:1014500002F01C06042202FA06F3234211D06B07A5
:101460000FD50B689B0603D40B6823F004030B60B5
:1014700090F8441001F01C018A40016C4A60016B35
:101480001DE0022303FA06F727424FF0000C4FF04D
:10149000010218D0AF0716D50C68A40605D40C6855
:1014A00024F00A040C6080F8252090F8441001F024
:1014B0001C018B40016C4B6080F824C0C16A00297C
:1014C0001AD0F0BC08470823B340234214D02B079E
:1014D00012D50B6823F00E030B6090F84410036CD8
:1014E00001F01C0102FA01F15960C26380F8252065
:1014F00080F824C0416BE2E7F0BC704770B568B17A
:101500002B4C036814212B4AA34209D22A4C1C44B9
:10151000B4FBF1F18900C0E910210BE0012070BD9E
:10152000234C64421C44B4FBF1F18900416420491E
:1015300008390164022180F825101C6847F6F07113
:101540008C43D0E902152943D0E904563543294399
:1015500085692943C5692943056A294321431960DF
:101560008168B1F5804F19D0036C0F21934202D1ED
:1015700052F8A83F02E00E4AA032136890F84440A7
:1015800004F01C04A1408B43136090F84430416880
:1015900003F01C0399401368194311600021C163D3
:1015A000012280F8252080F82410084670BD000034
:1015B0000804024000000240F8FFFDBF2DE9F05F83
:1015C000054632488946017801290CD0012680461B
:1015D00006704CF2503B5846FFF7A6F907004FF053
:1015E000000A03D04EE0022000F054B851464046B5
:1015F000C8F804A0264C226892050AD5216849053E
:1016000005D5216821F480612160032109E0067776
:1016100008E02268520504D5216821F48061216028
:10162000022101772868012807D04FF0FF31C9F85F
:10163000001040F2FA3BAE681DE06868FFF72EF933
:101640005846FFF771F90746606920F004006061B1
:1016500016E030466968FFF72FF94CF25030FFF77B
:1016600063F90700606920EA0B00606102D0C9F8E5
:10167000006005E0761CD5E902010844B042E8D8D4
:10168000FFF7DEF888F800A03846ADE744000020F8
:101690000020024030BCBDE8C09F00000348416903
:1016A00041F00041416100207047000000200240ED
:1016B0002DE9FF5F254C0646904620789A46012882
:1016C0000BD0012020704CF2503B5846FFF72CF90C
:1016D00007004FF0000904D02AE0022004B000F017
:1016E00039B84846C4F80490194D2968490504D50D
:1016F000286820F4806028600220207726B1012E1F
:1017000009D0022E07D00CE0424653460198FFF75D
:10171000E7F8012612E041460198FFF7EFF8022EA4
:101720000AD05846FFF700F94FEA0007FFF788F89C
:1017300084F800903846D1E74FF480265846FFF7EA
:10174000F3F807466869B0436861EFE7440000209A
:101750000020024030BCBDE8C09F000006490020C8
:101760004A69002A07DA054A8A60054A8A60496997
:10177000002900DA0120704700200240230167455C
:10178000AB89EFCD2DE9F04FDFF8AC9100230325B5
:10179000A9F1040B85B04FF0010C0F2709F1040AE1
:1017A000ABF1040EBFE000BF0CFA03F6324075D077
:1017B0000C7904F00304012C01D0022C1BD18468A5
:1017C00000945C0005FA04F80494009C24EA0804E0
:1017D0000094D1F80C80049C08FA04F8009C48EAB4
:1017E0000408C0F808804468B4430E79C6F30016B4
:1017F0009E40264346600C79E443A4070AD0C4689F
:101800004FEA430805FA08F6B4438E6806FA08F66C
:101810002643C6600C7904F00304022C10D1DC08C6
:1018200000EB84040294246A5E074FEAD66807FA44
:1018300008F6B4430E6906FA08F62643029C2662AF
:1018400004684FEA430805FA08F6B4430E7906F037
:10185000030606FA08F6264306604C6814F4403F77
:1018600060D0364C266E46F001062666246E23F0C4
:10187000030604F001040094314C34440294A4683B
:101880009E074FEA167807FA08F6B443B0F1904F76
:1018900005D02C4EB04204D1012612E042E00026D1
:1018A0000FE0294EB04201D102260AE0274EB04295
:1018B00001D1032605E0264EB04201D1042600E006
:1018C000072606FA08F62643029CA660D9F80060AF
:1018D0004C46D1F8048096435FEAC82800D51643E9
:1018E0002660DAF800405646D1F8048094435FEA57
:1018F000882800D514433460DBF800405E46D1F8F8
:10190000048094435FEA883800D514433460DEF8DD
:1019100000407646D1F8048094435FEAC83800D589
:10192000144334605B1C0A6832FA03F47FF43CAF62
:1019300005B000F00FB8000008040140001002409C
:10194000000001400004004800080048000C004866
:101950000010004830BCBDE8C08F0069084000D0CE
:10196000012070470AB181617047816270470000B1
:1019700001488068704700003800002002488168F4
:1019800002781144816070473800002010B50024AF
:10199000032000F09FF80F2000F008F808B10124A0
:1019A00001E000F04FF8204610BD000030B50546BC
:1019B0001F4887B0816D41F010018165806D06A9D7
:1019C00000F01000009001A800F0F6FA0498B0B101
:1019D00000F012FB40001749174AB0FBF1F117481D
:1019E000491E0260416040F2E7320021C0E9032154
:1019F0008160816101F056F8040003D015E000F029
:101A0000FBFAE8E70D4801F07FF804000DD136201D
:101A100000F032F8102D07D200222946362000F0BF
:101A200039F80748056000E0012407B0204630BDC2
:101A30000010024040420F0000100040C40200208D
:101A40003C0000200B4882B0016E41F001010166AC
:101A5000016E01F001010091816D41F080518165BD
:101A6000806D002200F0805000900F21901E02B087
:101A700000F010B800100240002809DB00F01F023F
:101A8000012191404009800000F1E020C0F80011E0
:101A900070470000F0B40E4B1B680C46C3F30223E2
:101AA000C3F10705042D00D90425191D072901D20A
:101AB000002300E0DB1E012606FA05F1491E214045
:101AC00099409E40761E16403143F0BC02F0ACBBFC
:101AD0000CED00E0064900F0070208684FF6FF032E
:101AE000184040EA0220034A104308607047000093
:101AF0000CED00E00000FA051649B0F5007F08681B
:101B0000C0F3412009D0022805D0086820F4C06045
:101B100040F480600860002070470128FBD008680E
:101B200020F4C06040F4007008600B483222006866
:101B300050430A4AB0FBF2F0401C00E0401E4A69E4
:101B4000520501D50028F9D148694005E3D50320A5
:101B500070470000007000406400002040420F0009
:101B60000B490A6822F00702921C0A6009490A68B8
:101B700042F004020A60012807D040BF20BF20BF06
:101B8000086820F004000860704730BFF8E70000E4
:101B90000070004010ED00E00248006800F4C060F2
:101BA00070470000007000400248016841F48071F5
:101BB00001607047007000402DE9F84F044600278F
:101BC0000088A84D3E46000515D5606C60B1B0F5A3
:101BD000000F04D0B0F5400F2BD001270AE0E868D1
:101BE00040F48030E86024E00021201D01F0DEFC9C
:101BF00007001ED03E46206880033AD5A86D4FF0FE
:101C00000008C00009D4A86D40F08050A865A86DF8
:101C10004FF0010800F080500090DFF84CA2DAF895
:101C2000001041F48071CAF80010FFF7A1FE814650
:101C300010E0D5F88800616C20F440000843C5F836
:101C40008800D8E7FFF794FEA0EB0900022801D92D
:101C5000032705E0DAF80000C005F3D5002F7DD09A
:101C60004FEA0706B8F1000F03D0A86D20F08050AE
:101C7000A8652078C00707D0D5F88800216A20F031
:101C800003000843C5F888002078800707D5D5F8F9
:101C90008800616A20F00C000843C5F888002078AD
:101CA000400707D5D5F88800A16A20F03000084326
:101CB000C5F888002078800607D5D5F88800E16A45
:101CC00020F440600843C5F888002088800507D5C7
:101CD000D5F88800E16B20F440200843C5F888005F
:101CE0002088400507D5D5F88800216C20F44010E5
:101CF0000843C5F888002078400607D5D5F8880045
:101D0000216B20F440500843C5F888002078000675
:101D100007D5D5F88800616B20F440400843C5F82A
:101D200088002088C00507D5D5F88800A16B20F46D
:101D300040300843C5F8880020684FF00067000372
:101D40004FF0806850D5D5F88800A16C20F0406035
:101D50000843C5F88800A06CB84200E005E03BD11C
:101D6000E86840F48010E8603EE0D5F8900010F498
:101D7000407014D0A16D814211D0D5F89000D5F8F3
:101D8000901020F4407041F48031C5F89010D5F8DF
:101D9000901021F48031C5F89010C5F89000C0076C
:101DA00011D0FFF7E5FD074641F2883907E000BF93
:101DB000FFF7DEFDC11B494501D9032652E7D5F8DF
:101DC00090008007F4D5D5F89000A16D20F4407004
:101DD0000843C5F8900045E7404505D10121201D85
:101DE00001F0E4FB00B106462068400317D5D5F8A2
:101DF0008800E16C20F040600843C5F88800E06C82
:101E0000B84204D1E86840F48010E86007E040453B
:101E100005D10121201D01F0C9FB00B10646208833
:101E2000400411D5D5F88800216D20F040500843BA
:101E3000C5F88800206DB0F1805F05D10221201D1A
:101E400001F0B4FB00B106462088000406D555F821
:101E5000880F616D20F0804008432860304600F014
:101E600005B80000001002400070004018BCBDE83A
:101E7000E08F00002DE9F0470F4605006BD0494E7A
:101E8000306800F00700B84209D2306820F007003F
:101E900038433060306800F00700B8425BD12878E2
:101EA000414C80070AD5A868A16801F0F00188427A
:101EB00004D9A16821F0F0010143A1602878C0078E
:101EC0002CD06868032811D0022812D0216898B15C
:101ED000490500293FDAA16821F003010143A1600F
:101EE000FFF746FD804641F2883910E021688901FC
:101EF000EFE721688903ECE78907EAE7FFF738FD98
:101F0000A0EB0801494502D90320BDE8F087A0688D
:101F1000696800F00C00B0EB810FEFD128788007E2
:101F20000AD5A868A16801F0F001884204D2A1682E
:101F300021F0F0010143A160306800F00700B842D1
:101F40000BD9306820F0070038433060306800F06B
:101F50000700B84201D00120D7E72878400705D50F
:101F6000A068E96820F4E0600843A06028780007D2
:101F700006D5A068296920F4605040EAC100A0603D
:101F800000F05EF8A168094AC1F30311515C01F049
:101F90001F01C8400649086006480068BDE8F047D0
:101FA000FFF704BD002002400010024088630008D3
:101FB000640000203C0000200F2202600C4A93685D
:101FC00003F003034360936803F0F00383609368B6
:101FD00003F4E063C36092684FF4E06303EAD20263
:101FE00002610448006800F00700086070470000C4
:101FF0000010024000200240054806490068896838
:10200000054AC1F30221515C01F01F01C84070472D
:102010006400002000100240C8630008054806491B
:1020200000688968054AC1F3C221515C01F01F01B3
:10203000C84070476400002000100240C8630008D8
:1020400070B52549002318468A68CC6812F00C0246
:1020500004F00306214C4FEA640509D00C2A05D090
:10206000042A32D0082A00D1284670BD012E10D192
:102070000B681B0704D4D1F89430C3F3032302E0A8
:102080000B68C3F30313164E56F82330DAB10C2A4B
:10209000EBD1C86800F00300022818D0032818D03C
:1020A0001846CA68CB68C2F30212C3F3062343433F
:1020B000521CB3FBF2F2C868C0F34160401C400000
:1020C000B2FBF0F070BD184670BD204670BD2046D2
:1020D000E7E72846E5E70000001002400024F4008E
:1020E000986300082DE9F84304006FD0FA4DA86802
:1020F00000F00C06E86800F003072078C00664D5FD
:1021000076B10C2E01D1012F0AD0A06900282868D1
:102110007AD040F001002860FFF72AFC80465DE09D
:102120002868800702D5A0690028DED0216A2868C7
:10213000000703D5286800F0F00004E0D5F894000B
:10214000F02202EA1010814216D9084601F0C4FAC2
:1021500000283BD1286840F0080028602868216AE0
:1021600020F0F000084328606868E16920F47F40AF
:1021700040EA0120686016E0286840F00800286006
:102180002868216A20F0F000084328606868E16947
:1021900020F47F4040EA0120686026B9206A01F0FF
:1021A0009BFA0028D5D1FFF74BFFA968CB4AC1F3B2
:1021B0000311515C01F01F01C840C9490860C948BA
:1021C0000068FFF7F3FB00287ED12EE0CAE000BFD5
:1021D000FFF7CEFBA0EB0800022876D8286880071E
:1021E000F6D5286840F0080028602868216A20F0A9
:1021F000F000084328606868E16920F47F4040EA05
:102200000120686011E0FFE720F001002860FFF77F
:10221000AFFB804606E000BFFFF7AAFBA0EB08007B
:102220000228DAD828688007F6D42078C00740D082
:10223000082E18D00C2E01D1032F14D06068B0F5F1
:10224000803F17D0B0F5A02F286817D020F4803039
:102250002860286820F4802028606068E0B1FFF7DB
:1022600087FB804614E02868800322D56068002838
:1022700078D01EE0286840F48030EDE740F48020FC
:102280002860F7E7FFF774FBA0EB08006428A4D8E8
:1022900028688003F6D50CE0FFF76AFB804605E06E
:1022A000FFF766FBA0EB0800642896D82868800337
:1022B000F6D4207880073BD5042E11D00C2E01D106
:1022C000022F0DD0E06801E0AAE1FFE000282868B5
:1022D0001ED040F480702860FFF74AFB07460CE0F0
:1022E000286840050CD5E0680028C1D008E000BF90
:1022F000FFF73EFBC01B022893D828684005F7D59E
:102300006868217C20F0F85040EA016068600FE0C6
:1023100020F480702860FFF72BFB074605E000BF24
:10232000FFF726FBC01B0228B1D828684005F7D468
:102330002078000729D560690028D5F8940012D0CC
:1023400040F00100C5F89400FFF712FB074604E0D7
:10235000FFF70EFBC01B022899D8D5F89400800720
:10236000F6D512E02BE120F00100C5F89400FFF74C
:10237000FFFA074605E000BFFFF7FAFAC01B022884
:1023800085D8D5F894008007F6D42078400766D524
:10239000A86D0027C00008D4A86D40F08050A86543
:1023A000A86D012700F0805000904F480168C905D2
:1023B00012D40168814641F480710160FFF7D8FAB8
:1023C000804605E0FFF7D4FAA0EB080002287DD88C
:1023D000D9F80000C005F5D5A068012816D0052859
:1023E000D5F8900017D020F00100C5F89000D5F87E
:1023F000900020F0040000BFC5F89000A06841F2F2
:102400008839C0B1FFF7B4FA80460FE0D5F89000E4
:1024100040F00100F0E740F00400C5F89000F5E757
:10242000FFF7A6FAA0EB080149454FD8D5F8900070
:102430008007F5D50EE0FFF79BFA804606E000BF67
:10244000FFF796FAA0EB080149453FD8D5F8900070
:102450008007F5D41FB1A86D20F08050A8652078C2
:10246000800628D5606A0028D5F8980012D040F080
:102470000100C5F89800FFF77BFA074605E000BFAA
:10248000FFF776FAC01B022820D8D5F898008007FD
:10249000F6D510E020F00100C5F89800FFF768FAC3
:1024A000074604E0FFF764FAC01B02280ED8D5F8EF
:1024B00098008007F6D4A06AF0B3022816D00C2E3C
:1024C0007DD0286820F08070286000E0A7E0FFF74A
:1024D0004FFA0446A6E0000000100240886300089E
:1024E000640000203C00002000700040E868E26AC0
:1024F00000F00301914228D1216B00F07002090124
:102500001039914221D1626B00F4FE41B1EB022FF0
:102510001BD194F8382000F07841B1EBC26F14D190
:10252000A18F00F4C00249084905A1F500119142AC
:102530000BD194F8401000E06AE04908490600F029
:10254000C060A1F1007181424BD00C2E73D028687D
:10255000400170D4286820F080702860FFF708FAE6
:10256000064604E0FFF704FA801B022857D82868C3
:102570008001F7D4F4E90B016FF00F0202EB0111B7
:102580000843218A5204490802EB4151A26841EAFA
:1025900002210843217D4FF07E42490802EB416150
:1025A0000843217B40EAC160E968244A114008439E
:1025B000E860286840F080702860E86800E03AE051
:1025C00040F08070E860FFF7D3F9044605E000BFF3
:1025D000FFF7CEF9001B022821D828688001F7D523
:1025E00027E02868800124D4286840F080702860A3
:1025F000E86840F08070E860FFF7BAF9044604E04C
:10260000FFF7B6F9001B022809D828688001F7D522
:102610000FE000BFFFF7ACF9001B022802D903202E
:10262000BDE8F88328688001F4D4E86804490840CC
:10263000E8600020F4E70120F2E700008C809D01B3
:10264000FCFFEEFE2DE9F047044690F8200001283B
:102650001ED0012684F82060022084F82100216821
:10266000CA2048622168532048622068816821F4AA
:10267000806181602068816821F480418160FFF77A
:1026800077F9054600274FF0FF084FF47A7911E0FB
:102690000220BDE8F08700BFFFF76AF9401B4845FC
:1026A00008D92168C1F82480032084F8210084F827
:1026B0002070EEE72068C0684007EDD52168C1F8BA
:1026C000248084F8216084F820700020E1E7000075
:1026D0002DE9F05F044690F8200093468A460128D1
:1026E00025D0012684F82060022084F8210021688A
:1026F000CA2048622168532048622068816821F41A
:10270000806181602068C16801F0800161F490619E
:10271000C1602068C0684FF0000740064FF0FF0816
:102720001AD4FFF725F905464FF47A7910E0022014
:1027300000F03CB8FFF71CF9401B484508D9216858
:10274000C1F82480032084F8210084F82070EFE78A
:102750002068C0684007EDD52168C1F814A0206842
:10276000816821F0070141EA0B0181600E48016890
:1027700041F4801101600C480830016841F4801177
:1027800001602068816841F480418160206881682F
:1027900041F4806181602168C1F8248084F821605F
:1027A00084F820700020C3E70004014030BCBDE87D
:1027B000C09F000004A001F013FD4FF40070FFF76C
:1027C0009BF901F041FD00005254432063616C6CA1
:1027D0006261636B0A00000010B50B4904464FF4B8
:1027E000801008602068C168490508D5C16801F0FB
:1027F000800161F49061C1602046FFF7DBFF01209A
:1028000084F8210010BD00001404014010B504003C
:102810004FF0010044D094F8210028B9002084F83A
:102820002000204600F040F8022084F821002168B2
:10283000CA204862216853204862204600F096FF73
:1028400000282DD120688168164A114081602168D6
:1028500088686268A369104322691A43104388603C
:102860002168E068086120680169228941EA024123
:102870000161204600F09EFF002811D12168CA6C3A
:1028800022F00302CA646269E16911432268D36CD1
:102890001943D1642268FF215162012184F821107B
:1028A00010BD0000BFFF8FFF10B598B004465C213B
:1028B0006846FDF744FD0F492068884218D14FF45F
:1028C00000300090401216906846FFF775F908B185
:1028D000FDF7B4FF084850F8901F41F40041016033
:1028E000002205210320FFF7D5F80320FFF7C4F8E5
:1028F00018B010BD002800400010024070B504461A
:1029000090F820000B4601281BD0012684F8206097
:10291000022084F82100B2B19878D97840EA0145C4
:1029200058781978000240EA413005432168CA20EE
:102930004862216853204862204600F017FFD0B15A
:1029400020E0022070BD5878C10603D500F0EF00EA
:102950000A305870D87800F0FDFE0504587800F071
:10296000F9FE45EA0025987800F0F4FE0543187852
:1029700045EA4035DAE708480540206845602046CA
:1029800000F018FF2268FF21516208B984F8216025
:10299000002184F8201070BD3FFFFF002DE9F041B9
:1029A000044690F8200090460D46012811D00127DA
:1029B00084F82070022084F821002168CA2048622F
:1029C000216853204862204600F0D0FE002618B14E
:1029D00029E00220BDE8F0812068B8F1000F80688E
:1029E0004FEA406024D0002800DBEE70A8782978F8
:1029F000EA7840EA01406978090241EA82510843D5
:102A000018490840216808602068816821F4802105
:102A10008160D5E90301084321688A681043886012
:102A2000204600F0C7FE2268FF215162A0B115E0E8
:102A3000002800DBEE70287800F08CFE0304687834
:102A400000F088FE43EA0023A87800F083FE0343E9
:102A5000E87843EA8050D3E784F8217084F8206056
:102A6000B8E700007F7F7F0070B504460068C1684A
:102A700021F0A001C160FEF77BFF05464FF47A7696
:102A800007E000BFFEF774FF401BB04201D90320EE
:102A900070BD2068C0688006F4D5002070BD704706
:102AA0007047704710B5040003D094F83D0010B192
:102AB00007E0012010BD002084F83C00204600F013
:102AC00022F8022084F83D00211D206801F0FCF866
:102AD000012084F8480084F83E0084F83F0084F820
:102AE000400084F8410084F8420084F8430084F8F0
:102AF000440084F8450084F8460084F8470084F8D0
:102B00003D00002010BD704790F83D10012901D014
:102B100001207047022180F83D100168CA6842F028
:102B20000102CA6000680B49884205D0B0F1804FAD
:102B300002D00949884207D18168084A1140062914
:102B400006D0B1F5803F03D0016841F0010101607A
:102B500000207047002C01400040014007000100A8
:102B6000704770B50446006801694FF00005C9431D
:102B7000890715D4C168C943890711D4E91E0161C9
:102B800001202077206880698007204602D0FFF767
:102B9000E7FF04E000F0A7F8204600F0A5F825774D
:102BA00020680169C943490717D4C168C943490767
:102BB00013D46FF00401016102202077206880693E
:102BC00010F4407F204602D0FFF7CAFF04E000F077
:102BD0008AF8204600F088F8257720680169C94303
:102BE000090716D4C168C943090712D46FF0080158
:102BF0000161042020772068C0698007204602D048
:102C0000FFF7AEFF04E000F06EF8204600F06CF82D
:102C1000257720680169C943C90617D4C168C9432B
:102C2000C90613D46FF010010161082020772068D5
:102C3000C06910F4407F204602D0FFF791FF04E006
:102C400000F051F8204600F04FF825772068016920
:102C5000C943C90708D1C168C943C90704D1891E3E
:102C60000161204600F042F820680169C943090665
:102C700009D4C168C943090605D46FF08001016118
:102C80002046FFF70DFF20680169C943C90509D433
:102C9000C168C943090605D46FF4807101612046FB
:102CA000FFF7FDFE20680169C943490609D4C168E0
:102CB000C943490605D46FF040010161204600F088
:102CC0001FF820680169C94389060BD4C168C9434C
:102CD000890607D46FF0200101612046BDE87040ED
:102CE000FFF7DFBE70BD7047704700000068034902
:102CF000884201D1FEF742BE70470000001000403C
:102D000070477047704770472DE9F04102680446EC
:102D1000D0691168936840F60F0528424FF000050E
:102D200005D186067ED58E067CD5616E1BE1994F56
:102D300003F001060F40374374D0C70709D0CF0511
:102D400007D501271762D4F8802042F00102C4F8A9
:102D5000802082070AD5DA0708D0276802223A6263
:102D6000D4F8802042F00402C4F8802042070AD53B
:102D7000DA0708D0236804221A62D4F8802042F0CF
:102D80000202C4F8802002070CD501F02002324371
:102D900008D0236808221A62D4F8802042F0080282
:102DA000C4F8802002050BD54A0109D523684FF4E9
:102DB00000621A62D4F8802042F02002C4F8802019
:102DC000D4F88020002A35D0800605D5880603D5A2
:102DD000616E09B120468847D4F88000216889686F
:102DE000490602D410F0280F26D0204601F03EF804
:102DF0002068806840061AD52068083050E8001F17
:102E000021F0400140E80012002AF5D1206F70B196
:102E100061498163206FFEF7EDFA00280AD0206F28
:102E2000816B01E00EE02046BDE8F04108472046F6
:102E3000FFF769FFBDE8F0812046FFF764FFC4F8A3
:102E40008050F7E7276E2026012F7BD1C70679D562
:102E5000CF0677D51020106220688068400641D5E3
:102E6000216F086840680004000CE3D0B4F85820D3
:102E70008242DFD9A4F85A000868006880062AD484
:102E8000206850E8001F21F4807140E80012002AF9
:102E9000F6D12068083050E8001F21F0010140E819
:102EA0000012002AF5D12068083050E8001F21F0F8
:102EB000400140E80012002AF5D1E6672566216846
:102EC00051E8000F20F0100041E80002002AF6D17E
:102ED000206FFEF76AFAB4F85800B4F85A10401A96
:102EE00081B22AE0B4F85800B4F85A10401A81B2FE
:102EF000B4F85A0000289DD000299BD0226852E8DF
:102F0000000F20F4907042E80003002BF6D12068F7
:102F1000083050E8002F22F0010240E80023002B87
:102F2000F5D1E66725666566226852E8000F20F055
:102F3000100042E80003002BF6D12046FFF7E1FE27
:102F400078E7FFE7C70209D55B0207D54FF4801089
:102F500010622046BDE8F041FFF7D4BE020606D558
:102F60000A0604D5A16E00297FF45DAF62E7400632
:102F7000E6D54806E4D52046026852E8001F21F055
:102F8000400142E80013002BF6D18667856600F009
:102F90000CF94FE720010004593E000810B5040069
:102FA00002D0A06F10B107E0012010BD002084F80E
:102FB0007400204600F026F82420A06720680168ED
:102FC00021F001010160204600F076FF0128ECD0DD
:102FD000606A10B1204600F0ADFE2068416821F41F
:102FE000904141602068816821F02A018160206859
:102FF000016841F0010101602046BDE8104000F089
:10300000FDBE00002DE9F0419EB00546142117A831
:10301000FDF795F95C216846FDF791F9314928687B
:1030200088425BD102260024684600960994FEF788
:10303000C3FD08B1FDF702FC2B48816D41F400315E
:103040008165816D01F400311C91C16C41F0010179
:10305000C164C06C17A900F001001C900C20CDE9E0
:1030600017060320CDE9194007201B904FF0904030
:10307000FEF788FB1E4F1D484FF080083860C7E9F7
:103080000164C7E903487C61BC61FC6138463C626D
:10309000FEF734FA08B1FDF7D1FB2F67BD62144F7C
:1030A000124848371430E7E802061020A7E811015B
:1030B0000F4847F814494830BC61FC613C62FEF798
:1030C0001DFA08B1FDF7BAFBEF66002205212620A4
:1030D000BD62FEF7DFFC2620FEF7CEFC1EB0BDE889
:1030E000F081000000440040001002406C000240EB
:1030F000340200202DE9F8430446806F1F4616462F
:103100000D4620284FD1CDB1C6B194F874000128E6
:1031100049D0012084F874004FF00008C4F8808082
:103120002120A067FEF724FCA4F850608146A4F893
:103130005260A068B0F5805F03D004E00120BDE8D4
:10314000F883206928B12E465FF0000584F874806A
:1031500010E00026FAE78021204600F0ADFFB8B964
:10316000C6B116F8010B21680885B4F85200401E5C
:10317000A4F85200B4F852004B464FF000020097FA
:103180000028E8D14FF04001204600F095FF30B113
:103190000320D4E735F8020BC0F30800E3E7202052
:1031A000A0670020CBE70220C9E77047FEE708B51B
:1031B000002100EB8000009101E0491C0091884251
:1031C000FBDC08BD2DE9F041002500F021FC0024C6
:1031D0004FF400764FF090474FF48068012231465B
:1031E0003846FEF7BFFB0220FFF7E1FF41463846B5
:1031F000FEF7B3FB40EA4500C5B20022314638462F
:10320000FEF7B0FB0320FFF7D2FF641CE4B2082CEA
:10321000E4D300F010FC2846BDE8F0812DE9F04130
:10322000054600244FF480684FF090474FF4007635
:10323000280601D5012200E0002241463846FEF76B
:1032400091FB012231463846FEF78CFB0220FFF746
:10325000AEFF002231463846FEF784FB0320FFF71D
:10326000A6FF6806641C050EE4B2082CE0D3BDE896
:10327000F08170B5012294024FF090452146284616
:10328000FEF770FB0122560231462846FEF76AFB24
:103290000320FFF78CFF002221462846FEF762FB41
:1032A0000320FFF784FF31462846BDE87040002226
:1032B000FEF758BB70B54FF480644FF09045002284
:1032C00021462846FEF74EFB012251022846FEF712
:1032D00049FB0220FFF76BFF012221462846FEF73B
:1032E00041FBBDE870400320FFF761BF70B50122CC
:1032F00094024FF0904521462846FEF733FB00F03C
:1033000087FB0122560231462846FEF72BFB06209A
:10331000FFF74DFF21462846FEF71FFB044600221B
:1033200031462846FEF71EFB00F085FB0CB100205D
:1033300070BD012070BD0000104810B50E4901603D
:103340000221416000214FF430228160C0E9031264
:103350004FF4001242610176012242768276C276F3
:1033600001774277FDF777FE002803D0BDE81040D3
:10337000FDF764BA10BD0000006400406401002045
:103380000D4808B5816C41F001018164806C002218
:1033900000F00100009005211020FEF77BFB1020BB
:1033A000FEF76AFB002205211120FEF773FBBDE842
:1033B00008401120FEF760BB0010024010B500F07D
:1033C000AFFA194C04202080184801F0A1FA174ADE
:1033D0000121E0611032084601F0CEFA134A206262
:1033E000303A0221102001F067FA104A6061183A61
:1033F0000221102001F060FA0C4AA0619C3A0021E1
:103400000B4801F005FB094AA060783A0021094801
:1034100001F0FEFA054AE060543A0021064801F046
:10342000F7FA206110BD0000040000206863000866
:1034300095390008993B0008AD060008F0B587B043
:1034400014216846FCF77BFF2448C16C41F004015D
:10345000C164C16C01F004010591C16C41F001012E
:10346000C164C16C01F001010591C16C41F0020120
:10347000C164C06C1A4E00F0020048F211040590BD
:10348000002221463046FEF76DFA4FF090470022A9
:103490004FF4E0613846FEF765FA0125CDE90045B5
:1034A00000240294694630460394FEF76BF9280223
:1034B0000090CDE90154694638460394FEF762F95D
:1034C0004FF4C06000901120CDE901040320039067
:1034D00069463846FEF756F907B0F0BD00100240C5
:1034E0000004004810B586B014216846FCF727FF99
:1034F0001D4800241B490594C0E900147F21816008
:10350000FF21C0E9031444618461C461FFF77EF9BF
:1035100008B1FDF793F915208DF800008DF80140F2
:103520008DF802400394012269460F480494FFF786
:1035300035FA08B1FDF782F901208DF814008DF8F5
:10354000150016208DF8160025208DF81700012291
:1035500005A90548FFF7D2F9002801D0FDF76EF95B
:1035600006B010BD002800408C0100200D4810B5A9
:103570000B4901604FF4E1314160002181600C2270
:10358000C160C0E904128161C16101624162FFF75B
:1035900005FD002803D0BDE81040FDF74FB910BD70
:1035A00000440040B0010020FEE7FEE72DE9F041B5
:1035B000444C05468846E0680026810728680DD0FF
:1035C000E16801F00301814216D1A8B1E0686968A1
:1035D000C0F30210401C88420ED120E0012804D024
:1035E000022805D0032807D108E02168890701E0F7
:1035F00021684905002907DB01265FE0216889036E
:1036000002D421684903F5E7E1686A686FF00F03A7
:1036100021F0730103EB021211430143E1602068C2
:1036200020F080602060FEF7A3F9074605E000BFA8
:10363000FEF79EF9C01B022837D820680001F7D496
:10364000B8F1000F18D0B8F1010F1DD0287D4FF050
:103650007E41400801EB4060A96840EA01202169F1
:10366000194A114008432061206840F080602060C2
:10367000FEF77EF907461AE0A868297B000240EAB7
:10368000C1602169114AECE7288A1149400801EB21
:103690004050A96840EA012021690E4AE1E700BFD5
:1036A000FEF766F9C01B022801D9032606E0206850
:1036B0000001F5D52069A969084320613046BDE8BD
:1036C000F081000000100240FF80FFF9FF80FF073B
:1036D0000000E0FFFF809FFFF8B51C4D0646002468
:1036E000A86DC00002D5FEF757FA0DE0A86D40F0B6
:1036F0008050A865A86D00F080500090FEF74CFA4D
:10370000A96D21F08051A965B0F5007F04D0802E0D
:1037100007D94FF003040AE0802E08D9A02E01D863
:1037200004E001D1022402E0702E00D101240848F7
:10373000016821F0070121430160006800F00700E3
:10374000A04201D00120F8BD0020F8BD00100240C9
:10375000002002400022014602E00A39C9B2521C90
:103760000A29FAD2100741EA106070472DE9F041AA
:10377000044600680025C168490617D4691EC16067
:10378000FEF7F6F806464FF47A78032708E000BF04
:10379000FEF7EEF8801B404502D9032584F821701E
:1037A0002068C068400601D4032DF1D12846BDE849
:1037B000F08100002DE9F04106461348002501681C
:1037C00021F080010160041F20684FF0030780068C
:1037D00007D43046FFF748F990B186F821700325E9
:1037E0000EE0206820F0200020603046FFF73CF912
:1037F00010B186F821700325206840F02000206079
:103800002846BDE8F08100000C2800400148FEF782
:10381000E3BF00008C010020F8B50026ADF8006081
:10382000684600F01CF9BDF8001023A000F0D8FC99
:10383000BDF80000FCF7A2FFBCEEC00A10EE100AB3
:1038400084B2214621A000F0CBFC26480088FCF77A
:1038500095FF00EE904AF8EE600A30EEC00ABDEE29
:10386000C00A10EE100A04B221461FA000F0B8FCF6
:10387000002C00DA00242348234D0088A04203DAFC
:1038800002202870012101E02E707821642000F0D0
:1038900033F9200A6870AC701CA000F0A1FC002471
:1038A0001DA0295D00F09CFC641C082CF8DB06A020
:1038B00000F096FCF8BD00005353435F526561640D
:1038C00044617461202564200A00000070726573F1
:1038D000737572655F70615F696E74202564200A7C
:1038E000000000000000002063616C696272617476
:1038F00065645F7072657373757265202564200A54
:1039000000000000060000202800002064617461AF
:103910005F5030313A20000025303258200000003E
:103920000B4802780B49FF2A02D14278FF2A06D0C1
:10393000028852BA0A808078FF2802D002E064220E
:10394000F8E71D208870C2B2098803A000F048BCC7
:1039500000FC0108060000204C6F6164656420646F
:103960006174613A207365636F6E645F7468726539
:1039700073686F6C643D2575202C2064656C6179DB
:103980005F726563656976656456616C75653D2532
:10399000750A00001CB5174F00254FF00108A94615
:1039A000A7F12C064FF4FA7AFFF736FFB08CB085FA
:1039B00096F8260086F82E000FA000F011FC0024D7
:1039C00010A0395D00F00CFC641C082CF8DB0FA083
:1039D00000F006FCCDE900892B4632880821054815
:1039E000FCF748FD6D1CEDB2FCF70EFF504600F0F1
:1039F00027FFD9E730000020646174615F503032E6
:103A00003A20000025303258200000000A00000053
:103A100000B585B014216846FCF791FC4FF4806036
:103A2000009000200190029069464FF09040FDF711
:103A3000A9FE05B000BD00B585B014216846FCF7AD
:103A40007EFC4FF4806000901120019000200290D5
:103A500069464FF09040FDF795FE05B000BD38B5C2
:103A6000044600200146009004236A46282000F006
:103A700097F89DF800109DF80120880901F03F019A
:103A800042EA0121218038BD1CB5002100918DF84A
:103A9000000001AB042269460648FDF711F818B191
:103AA00005A000F09DFB1CBD9DF800100BA000F0D0
:103AB00097FB1CBD008801084661696C6564207431
:103AC0006F2073617665204E4F44455F49442074F2
:103AD0006F20666C6173680A000000004E4F444519
:103AE0005F494420736176656420746F20666C6161
:103AF00073683A2025750A000EB50022030A019268
:103B00008DF804308DF805008DF806108DF807202B
:103B100002AB042201A90A48FCF7D2FF18B109A0A0
:103B200000F05EFB0EBD9DF8070000909DF806308A
:103B30009DF805209DF804100BA000F051FB0EBD70
:103B400000FC01084661696C656420746F20736134
:103B5000766520506172616D6574657220746F20A6
:103B6000666C6173680A0000506172616D6574650E
:103B70007220736176656420746F20666C6173686F
:103B80003A205B25755D205B25755D205B25755DA5
:103B9000205B25755D200A000A2000F051FEFBE73E
:103BA0002DE9F0411C4615460F460646FFF761FB1E
:103BB0007006000EFFF732FBFFF798FB00281ED0BF
:103BC0003846FFF72BFBFFF791FB002817D0FFF7D4
:103BD00050FB012000EB4600C0B2FFF71FFBFFF7D0
:103BE00085FB00280BD003E0FFF7ECFA05F8010B8A
:103BF000641EA4B2F8D2BDE8F041FFF75BBBBDE89C
:103C0000F08110B54FF0E020006902F0A9F9012819
:103C100003D0BDE8104001F05DBE10BD00B597B007
:103C200044216846FCF78BFB142111A8FCF787FBA5
:103C30004FF40070FDF760FF08B172B6FEE7FDF7C4
:103C4000B3FF194850F8901F21F0180101600E20B1
:103C5000012100900802CDE902101020CDE90401F5
:103C600002200A90CDE90B0108210D910721CDE931
:103C70000E1010906846FEF735FA08B172B6FEE7EE
:103C80000F20119003201290902013900020149088
:103C90000146159011A8FEF7EDF8002801D072B684
:103CA000FEE717B000BD00000010024002480168A6
:103CB00041F470010160704788ED00E00148FEF7B3
:103CC00050BF0000C402002070B50268164B4FF0D0
:103CD0008046984201D0B04203D122F070044A6875
:103CE0002243124C124D984205D0B04203D0A0425C
:103CF00001D0A84203D122F44076CA6832434E690B
:103D000022F08002324302608A68C2620A688262DC
:103D1000984203D0A04201D0A84201D109690163B1
:103D20000121416170BD0000002C014000400140B4
:103D30000044014090F82410C90706D001684A6881
:103D4000836A22F400321A434A6090F824108907EB
:103D500006D501684A68C36A22F480321A434A6071
:103D600090F82410490706D501684A68036B22F4CD
:103D700080221A434A6090F82410090706D501688A
:103D80004A68436B22F400421A434A6090F82410B8
:103D9000C90606D501688A68836B22F480521A43EB
:103DA0008A6090F82410890606D501688A68C36B7A
:103DB00022F400521A438A6090F82410490611D563
:103DC00001684A68036C22F480121A434A60016C4D
:103DD000B1F5801F06D101684A68436C22F4C00225
:103DE0001A434A6090F82410090606D501684A680B
:103DF000806C22F4002202434A607047F8B5002626
:103E00000446C0F88060FDF7B3FD054620680068F1
:103E10006FF07E47000708D52B4600224FF40011B3
:103E20002046009700F048F960B920680068400714
:103E30000AD52B4600224FF480012046009700F05F
:103E40003BF908B10320F8BD2020A067E067266693
:103E500084F874600020F8BD10B5806A0021A0F8D5
:103E60005A10A0F85210FEF74EFF10BD016851E83D
:103E7000002F22F4907241E80023002BF6D1016854
:103E8000083151E8002F22F0010241E80023002B05
:103E9000F5D1016E012908D1026852E8001F21F016
:103EA000100142E80013002BF6D12021C167002148
:103EB00001664166704700002DE9F0410446016843
:103EC00080682269E3691043626900251A43104340
:103ED000714F0A68714B1A4002430A6020684168BA
:103EE000E26821F44051114341602168A069B94260
:103EF00001D0226A10438A6822F4306202438A6049
:103F00006749236867488B420DD1D0F8880010F0CC
:103F1000030006D0012847D0022843D0032830D11F
:103F200044E001212EE060498B420BD1D0F888009B
:103F300010F00C0034D0042836D0082832D00C28D9
:103F40001FD133E059498B420BD1D0F8880010F0D3
:103F5000300025D0102827D0202823D0302810D199
:103F600024E0BB420DD1D0F8880010F4406017D097
:103F7000B0F5806F18D0B0F5006F13D0B0F5406F7A
:103F800014D010214A4A00264FF40040BB422FD1E2
:103F900071B102290FD004290FD0082973D10FE085
:103FA0000021EFE70221EDE70421EBE70821E9E733
:103FB000FEF722F803E0104602E0FEF741F8E8B30E
:103FC000626802EB420181425DD8B0EB023F5AD8F1
:103FD000010E03025008181871410023FCF762F922
:103FE000344AA0F5407191424DD82168C8604BE039
:103FF000E3694FF6EF77834228D1092943D2DFE8FE
:1040000001F005080B420D4242421000FDF7F4FF9B
:1040100006E0FEF703F803E0104602E0FEF710F8B2
:1040200060B14100606801EB5001B1FBF0F0A0F11C
:104030001001B94227D84FF6F07100E024E00140AA
:10404000C0F3420001432068C1601DE009291AD273
:10405000DFE801F005080B190D1919191000FDF71B
:10406000CBFF06E0FDF7DAFF03E0104602E0FDF7C4
:10407000E7FF48B1616800EB5100B0FBF1F0A0F13F
:104080001001B94205D9012566662846A666BDE835
:10409000F08180B2A9E7000000800040F369FFEFE3
:1040A0000038014000100240004400400048004039
:1040B0000024F400FFFC0F002DE9F0479A46174654
:1040C0000E4604464FF000094FF02008089D4AE0D4
:1040D000681C48D0FDF74CFCA0EB0A00A8422AD887
:1040E0004DB32068016849073DD5C069C04300054C
:1040F00039D421684FF400600862206850E8001F3E
:1041000021F4D07140E80012002AF6D1206808306E
:1041100050E8001F21F0010140E80012002AF5D10B
:10412000C4F87880C4F87C80C4F8808084F87490E7
:104130000320BDE8F087216851E8000F20F4D0701B
:1041400041E80002002AF6D12068083050E8001F3C
:1041500021F0010140E80012002AF5D1C4F878806E
:10416000C4F87C80E2E72068C06936EA000004D029
:104170000020B842ACD00020DBE70120F9E70000C6
:104180000148FEF7C1BD0000B0010020FEE70000BD
:1041900040F2FF610248018002A000F021B8000057
:1041A000000000205A65726F20506F696E742043C2
:1041B000616C6962726174696F6E20436F6D706CBF
:1041C000657465642E205A65726F204F666673654C
:1041D000743A2025642028726177290D0A000000B6
:1041E0000FB4054B10B503A9044A029800F04EF82D
:1041F00010BC5DF814FB000001470008E800002037
:104200000FB4084B10B504A902AA039800F03EF8B9
:10421000044602A9002000F06DFA204610BC5DF8AB
:1042200014FB0000F54600080907090E002804DB0E
:1042300000F1E02080F80014704700F00F0000F15A
:10424000E02080F8141D7047BFF34F8F05480168C8
:10425000054A01F4E06111430160BFF34F8F00BFD5
:10426000FDE700000CED00E00400FA0502E008C8DC
:10427000121F08C1002AFAD170477047002001E0E0
:1042800001C1121F002AFBD1704700002DE9FF4F2A
:104290008DB00F460546002606E025280BD0DDE947
:1042A0000F1290476D1C761C28780028F5D111B0AC
:1042B000304600F0F3B90024A246A1460122EC49A1
:1042C00000E0044315F8013F203B02FA03F00842E6
:1042D000F7D128782A2810D06FF02F022878A0F183
:1042E0003001092914D80AEB8A0102EB410144F09C
:1042F000020400EB010A6D1CF0E701CF5FEA000A3F
:1043000003D544F40054CAF1000A44F002046D1CC1
:1043100028782E2817D115F8010F44F004042A2814
:104320000ED06FF02F022878A0F1300109290AD8A9
:1043300009EB890102EB410100EB01096D1CF2E779
:1043400057F8049B6D1C28786C280FD006DC4C288D
:1043500017D068280DD06A2814D104E0742810D032
:104360007A280FD10DE044F400140AE044F48014DC
:1043700001E044F440146978814202D104F58014CC
:104380006D1C6D1C2A786E2A1FD00CDC632A31D07C
:1043900004DC002A8BD0582A11D1A3E0642A68D00B
:1043A000692A0CD165E0732A2ED004DC6F2A73D001
:1043B000702A04D19BE0752A6FD0782A6ED01046FF
:1043C000DDE90F129047761C50E1C4F30250022839
:1043D00006D0032809D0042801CF09D0066045E1A2
:1043E00001CFF117C0E9006140E101CF06803DE156
:1043F00006703BE117F8040B8DF8000000208DF8E3
:104400000100EB46012003E057F804BB4FF0FF30FA
:1044100061074FF0000102D40DE008F10101884668
:1044200049450FDA8045F8DB1BF808100029F4D164
:1044300008E008F1010188468142FADB1BF8081008
:104440000029F6D1DDE90F23AAEB080081462146B9
:1044500000F039F9304400EB080604E0DDE90F1202
:104460001BF8010B9047B8F10108F7D221464846E6
:10447000F7E00A21C4F302534FF0000B0891022B1E
:1044800004D001CFC117032B09D00AE0FF1D27F08C
:104490000707F7E8020108E032E01FE020E000B281
:1044A000C117042B01D140B2C117031E71F10003E3
:1044B00007DA4FF0000CD0EB0C006CEB01012D2360
:1044C00002E0230504D52B238DF82430012303E0DB
:1044D000E30701D02023F7E7984658E00A2110E0CF
:1044E00010210EE010204FF0000B08900CE010217E
:1044F0004FF0000B44F004044FF00809089103E06A
:1045000008214FF0000B0891C4F30253022B04D092
:1045100001CF0021032B06D006E0FF1D27F007077F
:10452000F7E8020103E080B2042B00D1C0B24FF0E3
:10453000000823072BD5702A07D0DDF820C08CF0A7
:10454000100C5CEA0B0C05D00EE040238DF82430F3
:10455000012308E050EA010306D030238DF824300F
:104560008DF8252002239846DDF820C08CF0080C39
:104570005CEA0B0C0BD150EA010301D1630706D5AD
:1045800030238DF824304FF00108A9F10109582A91
:1045900004D038A20B9208AA0A920BE03AA2F9E7DB
:1045A0005B46089AFBF77EFE0B9B9B5C0A9A521EA9
:1045B0000A92137050EA0102F2D10A98ADEB0000A2
:1045C00000F1200B600702D524F4803401E04FF0A5
:1045D0000109D94502DDA9EB0B0000E0002000EB4A
:1045E0000B0141440890AAEB010AE00306D4DDE97F
:1045F0000F232146504600F066F806444FF00009AC
:1046000008E009A911F80900DDE90F12904709F146
:104610000109761CC145F4DBE0030CD5DDE90F236D
:104620002146504600F04FF8064404E0DDE90F1241
:1046300030209047761C0899481E08900029F5DC28
:1046400008E00A980A990078491C0A91DDE90F12DE
:104650009047761CBBF10001ABF1010BF1DC214668
:104660005046DDE90F2300F01CF806446D1C1BE6E4
:104670000928010030313233343536373839616238
:1046800063646566000000003031323334353637FC
:1046900038394142434445460000000030BCBDE883
:1046A000C08F2DE9F041044600251E4617468804B8
:1046B00004D405E039462020B0476D1C641EF9D5AE
:1046C0002846BDE8F0812DE9F041044600251E464C
:1046D0009046C80301D5302700E02027880404D580
:1046E00005E041463846B0476D1C641EF9D52846A2
:1046F000BDE8F0810A68531C0B6010707047000021
:1047000013B54FF47A73012269460248FEF7F2FCB2
:1047100000981CBDB001002010B5002821D0114B1D
:104720000022001F196803E0814203D80A46496845
:104730000029F9D152B11368841A9C4204D100684F
:1047400018441060104602E0506000E0186039B173
:1047500002680B1A934203D10B681A44026049683D
:10476000416010BDEC000020FDF710F9FFF756FA8C
:10477000FEF764FEFEF704FEFEF7DEFDFEF7F6FE32
:10478000FEF7B0FE0AA0FFF72BFDFBF72FFE104847
:10479000FCF7D8FD02210E48FCF7FDF9FFF7F8FC05
:1047A00000F05CF8FEF70AFE00F06AF8FEE7000091
:1047B000486F6E657965656C6C5F50726573737573
:1047C000726520323032355F345F330D0A000000ED
:1047D00064010020F0B50B30154D20F007010024D6
:1047E000144A0FE003688B420BD38B4205D95E1A43
:1047F00043184768C3E9006700E04368136002C0DC
:1048000004E0021D10680028ECD12046002802D1E7
:10481000286808B10020F0BD064A07481060074A22
:10482000121A22F00702C0E9002401202860D7E70D
:10483000F0000020EC000020EC4F0020E8510020A8
:1048400010B5EFF3058111B16FF0050403E000240A
:1048500008B100F0DFFE204610BD0000EFF3058038
:1048600010B16FF0050070470448016811B14FF0B6
:10487000FF3070470121016000207047B800002020
:1048800010B5EFF3058010B16FF0050010BD0848BA
:104890000168012902D04FF0FF3010BD054A002108
:1048A00082F8141D0221016000F01CFF002010BDE1
:1048B000B80000200BE000E0F8B514464FF000050A
:1048C000EFF3058212BB08B301B3A4B1D4E90232FD
:1048D00063B1502A1AD32269C2B1676900FB01F69D
:1048E000B74213D3009501F081F807E072B922694D
:1048F00062B9626952B9002201F057F8050005D08B
:104900000CB1216800E0002100F022FE2846F8BD2D
:1049100070B505464FF00004EFF3058050BB0DB1B4
:10492000686800E00020C10701D0012600E00026F1
:1049300000071FD46DB1D5E9021021B1502819D359
:104940001EB1042002E020B114E0012001F020F8A3
:1049500005E00EB1042000E0012001F00EF8040093
:1049600008D00DB1296800E0002100F0F1FD0EB182
:1049700044F00104204670BDF8B5144603460E46C7
:104980004FF00005EFF3058098BB93B39E423DD8EE
:104990004CB1A0680028E06803D0502836D301202D
:1049A00002E008B132E00020012B05D010B3184618
:1049B000A26800F0C2FF20E040B103200090002276
:1049C00011460120A36801F011F804E00322002140
:1049D000012000F0EAFF050018D086B100231A4636
:1049E000194601F07BF8012809D0284600F0C4FDE3
:1049F00000250BE0184600F083FF050006D00CB13F
:104A0000216800E00021284600F0A2FD2846F8BDFC
:104A10002DE9FF410B464FF00005EFF305810395AB
:104A200049BB40B38027182100244AB3166806B159
:104A3000344696691EB13146761E382E02D216795A
:104A4000F60703D0002004B0BDE8F081566906B136
:104A5000B708D2F808C0BCF1000F0DD0D5685C2DA6
:104A600018D312693AB136B18DE806103A4621469C
:104A700001F04AFA03900DE0D6685EB912694AB9AE
:104A800003AACDE90012BAB2214601F00DFA0128BD
:104A900000D003950398D6E72DE9F041134C0F465B
:104AA0000546E6682068001D00F054FC681C07D12C
:104AB00037B12168BDE8F0410D48091D00F09ABCEE
:104AC00020683544B5424560216805D2A06BBDE839
:104AD000F041091D00F076BC606B091D00F072FC0E
:104AE000A06A854200D2A562BDE8F081680000207E
:104AF000000800202DE9F041054600F087FC2D4C10
:104B0000A068401CA06020682B4F10B1606930B3D2
:104B10002BE02560A068012827D1002606EB86003F
:104B200007EB800000F040FC761C382EF6D32348BB
:104B300000F03AFC2148143000F036FC1F482830C1
:104B400000F032FC1D483C3000F02EFC1B48503079
:104B500000F02AFC194860631430A06305E0206867
:104B6000E96AC06A884200D82560606A401C6062B9
:104B70006864E86A2169884200D9206100EB8000FE
:104B800007EB8000291D00F035FC00F05FFC606938
:104B900000280CD02068E96AC06A884207D2084918
:104BA0004FF080500860BFF34F8FBFF36F8FBDE8A9
:104BB000F08100006800002050030020B0070020B2
:104BC00004ED00E038B500F021FC104C2068C8B9B5
:104BD0000F4800F0E9FB0E48143000F0E5FB0C48EC
:104BE000E060143020610A4B0020F03B009003F19C
:104BF000500210210A2000F0F9FE206010B105A13A
:104C000000F0A6FCBDE8384000F020BCA400002065
:104C100004090020546D72510000000030B4026C91
:104C20000B46002A0BD0C1681144C1608468A142C0
:104C300001D30168C16030BC1846FBF767BB30BCCC
:104C400070472DE9F041856B174604460026026C3B
:104C500082B1C7B1E068FBF759FBE168206C091A23
:104C6000E1602268914202D2A168081AE060022F36
:104C700016D017E02068A8B9A06801F0E9F9064647
:104C80000020A0600EE06068FBF740FB216C6068CC
:104C900008446060A168884204D32068606001E035
:104CA00005B16D1E6D1CA5633046BDE8F08110B5E1
:104CB000044690F8590058B101280CD002280FD0B2
:104CC000502080F31188BFF34F8FBFF36F8FFEE743
:104CD000206B00F0CFFB2046BDE8104000F0CABBBF
:104CE00010BD000010484FF48041420706D0C01D9F
:104CF0000D4920F00700411AC1F580410B4A0023FD
:104D00000144C2E900030839183A21F00701116093
:104D10004B600B600B1AC0E9001393604FF000402A
:104D20005360506170470000E40F0020D400002061
:104D3000144E154CA6F29C474FF08058DFF84C906B
:104D400012E000BF00F062FBF068C568281D00F0AB
:104D500001FBA068401EA0606068401E606000F01B
:104D600075FB2846FFF7A3FF60680028EAD1386882
:104D70000128F9D9C9F80080BFF34F8FBFF36F8FB7
:104D8000F2E70000EC0700206800002004ED00E0DE
:104D9000002807D00021816001600B460A46C160EF
:104DA00000F09CBE7047000070B51D46049C51B1D8
:104DB000C4F80020C4E90F010121204600F04AFE9A
:104DC00084F84C5070BD2460F4E700002DE9F05FDA
:104DD0008846DDE90B941546834691009A460A9E63
:104DE000A522206BFBF7A4FA6FF00301206B01EB07
:104DF0008501084420F00707780707D0502080F38A
:104E00001188BFF34F8FBFF36F8FFEE70025B8F116
:104E1000000F0FD05FF00000221818F8001082F881
:104E2000341018F8001011B1401C1028F4D384F885
:104E3000435001E084F83450382E00D33726E66220
:104E4000C4E91365201D00F0BAFA04F1180000F05F
:104E5000B6FA2461C6F138006462A061656584F821
:104E6000585052465946384600F05EFA2060B9F173
:104E7000000F01D0C9F8004000F000B830BCBDE818
:104E8000C09F000030B5114900E011460A68824217
:104E9000FBD34B685C18844203D1406818444860D7
:104EA000084643681C18944209D1084C183C2468F1
:104EB000A24209D052681A4442600A68126802602D
:104EC000814200D0086030BD0460F9E7D4000020C2
:104ED00070B5002441600B4D0061914206D8D11A93
:104EE0008269914206D2011D286907E09A4203D2E5
:104EF000994201D3012403E0011DE86800F062FA41
:104F0000204670BDA400002010B5044600F07EFAD3
:104F1000A06B28B15FF0000400F098FA204610BDA5
:104F20000124F9E730B589B03C4D6EE004980028C3
:104F300006DADDE90601059A90470498002864DB4B
:104F4000069C606910B1201D00F004FA03A800F06F
:104F5000D7F8024604980A2857D2DFE800F0050582
:104F6000052D334A05052D3394F8280040F0010043
:104F700084F828000599A069059B01442046FFF7A5
:104F8000A7FF68B3216A2046884794F828004007A5
:104F90003BD5002000900598A169002342181946CE
:104FA000204601F05FF9D8B9502080F31188BFF393
:104FB0004F8FBFF36F8FFEE714F8280F20F001002A
:104FC000207022E094F8280040F0010084F82800C6
:104FD0000598A06128B1811813462046FFF778FF95
:104FE00013E0502080F31188BFF34F8FBFF36F8F12
:104FF000FEE794F82800810703D4204600F03AFA2F
:1050000003E020F0010084F82800002204A92868A9
:1050100000F074FE002889D109B030BDA400002042
:105020002DE9FC410F46054600F0A0FB01A800F069
:1050300067F80446019818B101F082F8BDE8FC81D8
:10504000254EAFB130690068D0B30027291B3A461E
:10505000306800F0BDFA01F073F80028EED11F4966
:105060004FF080500860BFF34F8FBFF36F8FE5E7BD
:10507000A542EBD801F064F8F0682746C068C46820
:10508000201D00F067F994F82800410719D5A069A0
:105090002B4641193A462046FFF71AFFA8B10020D7
:1050A0000346014600902A46204601F0DBF860B92D
:1050B000502080F31188BFF34F8FBFF36F8FFEE74F
:1050C00007E020F0010084F82800216A2046884784
:1050D000B4E70127BAE70000A400002004ED00E0D7
:1050E0000648416B096829B1416BC968C9684968BC
:1050F000816270474FF0FF31FAE70000680000203E
:1051000070B5054600F03AFF064E0446B06884428A
:1051100003D200F009F8012000E0002028602046BA
:10512000B46070BDA4000020F8B5194D20E0C0683F
:10513000C4680668201D00F00DF9216A20468847E2
:1051400094F82800400713D5A0693044B04206D92E
:1051500024616060211DE86800F034F908E0002057
:105160000346014600903246204601F07BF838B1F4
:10517000E86801680029DAD12969C5E90310F8BD9A
:10518000502080F31188BFF34F8FBFF36F8FFEE77E
:10519000A400002008484068401C4FF0500080F3F5
:1051A000118804D0BFF34F8FBFF36F8FFEE7BFF3BB
:1051B0004F8FBFF36F8FFEE7DC000020074CE068E5
:1051C000016841B1C0680021D0F80000FFF728FF56
:1051D000FFF7A8FEF3E701210020F7E7A400002075
:1051E0002DE9F041044600F011F994F9455004F11D
:1051F000240609E0606A48B1304600F069FF08B152
:1052000000F036FA6D1E6DB2002DF3DC4FF0FF3664
:1052100084F8456000F01AF900F0F8F894F9445069
:1052200004F1100709E0206948B1384600F050FF4A
:1052300008B100F01DFA6D1E6DB2002DF3DC84F88C
:105240004460BDE8F04100F001B900002DE9F041F3
:105250000546002700F08AFA324E306808B9FFF799
:1052600041FD706905424ED1C5B3083568070ED0BF
:1052700005F00700C0F108000544680707D050207A
:1052800080F31188BFF34F8FBFF36F8FFEE72DB30D
:105290007068854237D82348183001460C6801E011
:1052A00020460C466168A94202D221680029F7D144
:1052B00031688C4227D00768216801606068083730
:1052C000411B10290FD96019420708D0502080F3E4
:1052D0001188BFF34F8FBFF36F8FFEE713E041607C
:1052E0006560FFF7CFFD61687068401A7060B26852
:1052F000904200D2B060706901430020C4E900010F
:10530000F068401CF06000F01BFF780707D05020C9
:1053100080F31188BFF34F8FBFF36F8FFEE73846DE
:10532000BDE8F081BC00002010B5031F4FF0807471
:105330001C601B1F21F001011960191F044B0B6039
:1053400014390A60091F6FF0020244380A6010BD68
:1053500095510008D0E9013201699A60D0E9012332
:105360005A604A68824201D182684A600022026122
:105370000868401E0860086870470000034B03601F
:1053800003F15C0008608020106070472C09002049
:10539000044B036003F15C0008604FF48070106000
:1053A00070470000880B002000F108014FF0FF3229
:1053B000C0E90112C1600161002101607047002154
:1053C0000161704730B50B685A1C02D000F1080229
:1053D00002E0026904E02246546825689D42FAD939
:1053E00053684B6099608A60516008610168491C8C
:1053F000016030BD42684A6093688B609368596071
:10540000916008610168491C01607047502080F379
:105410001188BFF34F8FBFF36F8F0A494868401C54
:10542000486001280CD10848006810F0FF0F07D031
:10543000502080F31188BFF34F8FBFF36F8FFEE7CB
:1054400070470000DC00002004ED00E008494868D7
:1054500028B1401E486001D180F311887047502068
:1054600080F31188BFF34F8FBFF36F8FFEE700000B
:10547000DC00002070B500282AD0164DA0F10804E9
:1054800060686969084207D1502080F31188BFF332
:105490004F8FBFF36F8FFEE722683AB1502080F341
:1054A0001188BFF34F8FBFF36F8FFEE788436060B3
:1054B00000F05CF960686968084468602046FFF79E
:1054C000E1FC2869401C2861BDE8704000F038BE4E
:1054D00070BD0000BC0000204FF0E0200021016101
:1054E000816105494FF47A720968B1FBF2F1491EF6
:1054F00041610721016170476400002010B5FAF78F
:10550000ABFE114910280ED300F1E02090F8F00313
:105510000A78904207D2502080F31188BFF34F8F52
:10552000BFF36F8FFEE709480068896800F4E06008
:10553000884207D9502080F31188BFF34F8FBFF303
:105540006F8FFEE710BD0000DC0000200CED00E0D6
:1055500010B5084B002200BF53F832401CB1521C5A
:10556000082AF9D310BD43F8321003EBC20148609A
:1055700010BD00001003002010B504000AD000F098
:1055800013F894F8460000280CD12046BDE81040DE
:10559000FFF770BF502080F31188BFF34F8FBFF328
:1055A0006F8FFEE710BD0000084A002102EBC10327
:1055B0005B68834206D1002042F8310002EBC10152
:1055C00048607047491C0829F0D370471003002039
:1055D00070B515460E460446FFF718FF94F94410BF
:1055E0000020491C01D184F8440094F94510491C5D
:1055F00001D184F84500FFF729FFA06B28B92A469E
:10560000314604F1240000F051F82046BDE8704016
:10561000FFF7E6BD10B5020014D00F48006B38B19B
:10562000502080F31188BFF34F8FBFF36F8FFEE7D9
:1056300000F09CF800211046FFF72EFA00F080FDE4
:10564000002807D105494FF080500860BFF34F8F05
:10565000BFF36F8F10BD00006800002004ED00E074
:1056600002490A6A0260C968416070476800002008
:1056700001490120C86170476800002010B50C4640
:1056800050B1094909681831FFF79CFE2046BDE872
:1056900010400121FFF700BA502080F31188BFF3BA
:1056A0004F8FBFF36F8FFEE76800002070B5144680
:1056B0000D4668B10A4909681831FFF79BFE0CB125
:1056C0004FF0FF3521462846BDE87040FFF7E4B9AA
:1056D000502080F31188BFF34F8FBFF36F8FFEE729
:1056E0006800002030B587B00024039405AA04A9FF
:1056F00003A80494FFF742FEDDE903010094CDE91D
:105700000110002315A11748059A00F0FDFB164D66
:105710000028E8621FD000F075FD012809D0401C68
:1057200019D1502080F31188BFF34F8FBFF36F8FD3
:10573000FEE7502080F31188BFF34F8FBFF36F8FC8
:105740004FF0FF30A86201206861EC6007B0BDE84F
:10575000304000F045B807B030BD000049444C452A
:1057600000000000314D0008680000200248016B75
:10577000491C01637047000068000020164810B5FE
:10578000016B11B10121C16110BD0021C16101692D
:10579000124A01E0B9B1491E01EB810352F82330EE
:1057A000002BF7D001EB810302EB830202F1080426
:1057B00053685B685360A34201D15B685360DA6849
:1057C0000260016110BD502080F31188BFF34F8F3C
:1057D000BFF36F8FFEE70000680000205003002039
:1057E0001CB537480168374A914207D1502080F3F1
:1057F0001188BFF34F8FBFF36F8FFEE70068314909
:10580000491E884207D1502080F31188BFF34F8F83
:10581000BFF36F8FFEE72C4908780190FF200870D6
:1058200008788DF800009DF800009DF8002000F039
:10583000F000904207D0502080F31188BFF34F8FC3
:10584000BFF36F8FFEE79DF80000204C00F0500082
:1058500020700720A06005E09DF8002052008DF820
:105860000020401E9DF800201206F5D4A0600328F9
:1058700007D0502080F31188BFF34F8FBFF36F8F95
:10588000FEE74FF44070A060019808700C4820308B
:10589000016841F470010160016841F070410160EC
:1058A000FFF71AFE00206060FAF79EFC08480168C6
:1058B00041F040410160FAF783FC00201CBD00006C
:1058C00000ED00E071C20F4100E400E0DC000020C8
:1058D00034EF00E010B5502080F31188BFF34F8FF4
:1058E000BFF36F8F00F050FB18B104494FF08050A8
:1058F0000860002080F3118810BD000004ED00E076
:1059000010B50C4648B184420FD9502080F311885D
:10591000BFF34F8FBFF36F8FFEE7502080F31188E6
:10592000BFF34F8FBFF36F8FFEE70222002100F01D
:105930003CF8002800D0846310BD38B50C4648B14F
:1059400084420FD9502080F31188BFF34F8FBFF3EB
:105950006F8FFEE7502080F31188BFF34F8FBFF3A6
:105960006F8FFEE70221134600220091114600F0DE
:105970003DF8002800D0846338BD10B502460021F0
:10598000012000F012F80446FFF702FA204610BD8D
:1059900038B50B46002200901146012000F026F891
:1059A0000446FFF7F5F9204638BDF8B517460E4610
:1059B000050013D005FB06F05030FFF747FC04004C
:1059C0000AD0002084F8460004F150023B463146DC
:1059D00028460094FFF7E8F92046F8BD502080F3F0
:1059E0001188BFF34F8FBFF36F8FFEE738B5049D6B
:1059F00018B153B1CAB181B120E0502080F31188B1
:105A0000BFF34F8FBFF36F8FFEE7502080F31188F5
:105A1000BFF34F8FBFF36F8FFEE7502080F31188E5
:105A2000BFF34F8FBFF36F8FFEE739B1502080F384
:105A30001188BFF34F8FBFF36F8FFEE750241C46D2
:105A4000012384F846302B460094FFF7ADF9204639
:105A500038BD000070B50D46040025D0FFF7D6FC18
:105A6000D4E90F20216802FB0011A1600021A1638D
:105A7000216861600A46D4E90F01401E00FB012144
:105A8000E16021464FF0FF3001F8440F487004F107
:105A900010008DB1FFF788FC04F12400FFF784FCAF
:105AA000FFF7D4FC012070BD502080F31188BFF3B4
:105AB0004F8FBFF36F8FFEE721690029F0D000F010
:105AC00007FB0028ECD004494FF080500860BFF37A
:105AD0004F8FBFF36F8FE3E704ED00E02DE9FF4741
:105AE00082B01D468A464FF00008040003D0BAF188
:105AF000000F08D011E0502080F31188BFF34F8FC2
:105B0000BFF36F8FFEE7206C38B1502080F311880F
:105B1000BFF34F8FBFF36F8FFEE7022D0AD1E06B0B
:105B2000012807D0502080F31188BFF34F8FBFF3B7
:105B30006F8FFEE700F014FA3F4F4FF000094FF06F
:105B4000805648B9049838B1502080F31188BFF3CB
:105B50004F8FBFF36F8FFEE7FFF758FCA06BE16B31
:105B6000884207D3022D05D00498D0B1B8F1000FB8
:105B70001AD01EE02A4651462046FFF762F8616AB5
:105B800019B104F1240000F0A3FA20B13E60BFF384
:105B90004F8FBFF36F8FFFF759FC012006B0BDE8B0
:105BA000F087FFF753FC22E06846FFF759FD4FF0FE
:105BB0000108FFF74BFCFFF7D9FDFFF727FC94F92D
:105BC0004400401C01D184F8449094F94500401CE5
:105BD00001D184F84590FFF739FC04A9684600F02C
:105BE00029F930B12046FFF7FBFA00F0A9FA0020AE
:105BF000D4E7FFF70BFCA06BE16B884213D1FFF7F2
:105C000025FC04F110000499FFF738FD2046FFF74A
:105C1000E7FA00F095FA00289ED13E60BFF34F8F5F
:105C2000BFF36F8F98E7FFF711FC2046FFF7D8FA14
:105C300000F086FA90E7000004ED00E02DE9F0475F
:105C40001F4690468946040003D0B9F1000F08D0E2
:105C500011E0502080F31188BFF34F8FBFF36F8F97
:105C6000FEE7206C38B1502080F31188BFF34F8FCE
:105C7000BFF36F8FFEE7022F0AD1E06B012807D038
:105C8000502080F31188BFF34F8FBFF36F8FFEE773
:105C9000FFF734FC5020EFF3118680F31188BFF337
:105CA0004F8FBFF36F8FA06BE16B884206D3022F3B
:105CB00004D0002086F31188BDE8F08794F94550A0
:105CC000A06B3A4649462046FEF7BBFF681C04D04D
:105CD0006D1C84F845500120ECE7606A0028FAD07A
:105CE00004F1240000F0F4F90028F4D0B8F1000F1A
:105CF000F1D00121C8F80010EDE700002DE9F747C9
:105D0000002683B08A46040003D0BAF1000F08D001
:105D100011E0502080F31188BFF34F8FBFF36F8FD6
:105D2000FEE7206C38B1502080F31188BFF34F8F0D
:105D3000BFF36F8FFEE700F013F9DFF8F4804FF048
:105D400000094FF0805748B9059838B1502080F3CA
:105D50001188BFF34F8FBFF36F8FFEE7FFF756FB3E
:105D6000A56BC5B151462046FEF758FF6D1EA563D1
:105D7000206950B104F1100000F0AAF928B1C8F868
:105D80000070BFF34F8FBFF36F8FFFF75FFB0120F2
:105D900006B0BDE8F087059808B11EB106E0FFF730
:105DA00055FB27E06846FFF75BFC0126FFF74EFB3B
:105DB000FFF7DCFCFFF72AFB94F94400401C01D1FB
:105DC00084F8449094F94500401C01D184F8459032
:105DD000FFF73CFB05A9684600F02CF80028204698
:105DE0000AD0FFF7FDF900F0ABF92046FFF78CF879
:105DF0000028B3D00020CBE7FFF786F890B104F17C
:105E000024000599FFF73AFC2046FFF7E9F900F076
:105E100097F90028A2D1C8F80070BFF34F8FBFF3E5
:105E20006F8F9BE72046FFF7DBF900F089F995E7D4
:105E300004ED00E02DE9F0410C46050011D0C4B19D
:105E4000FFF7E4FA174BDA686E682068911B471C6D
:105E500017D02F681B6A9F4219D0964217D8012489
:105E600010E0502080F31188BFF34F8FBFF36F8F86
:105E7000FEE7502080F31188BFF34F8FBFF36F8F81
:105E8000FEE70024FFF7E2FA2046BDE8F0818842F1
:105E900005D9401A20602846FFF7E2FBF1E7002011
:105EA0002060DCE7680000202DE9FF5F8346DDE924
:105EB0000E87994616468A469000FFF7C7F90500F7
:105EC0001CD05C20FFF7C2F9040014D00020256329
:105ED00084F85900CDE90240CDE900874B463246AF
:105EE00051465846FEF772FF2046FEF703FE01209A
:105EF00004B000F006B82846FFF7BCFA4FF0FF30B8
:105F0000F6E730BCBDE8C09FF0B585B0DDE90B64B5
:105F10000A9DA6B1DCB15C2700972663022684F8AF
:105F20005960002604AFCDE90246CDE90057FEF7DF
:105F30004DFF2046FEF7DEFD049805B0F0BD502071
:105F400080F31188BFF34F8FBFF36F8FFEE75020B0
:105F500080F31188BFF34F8FBFF36F8FFEE7000010
:105F60000548416919B1006B18B100207047012044
:105F70007047022070470000680000200148C06898
:105F800070470000680000202DE9F0412E4C0027EA
:105F9000206B28B1A069401CA0613846BDE8F081A3
:105FA000E668761CE66013D1606B006838B150205B
:105FB00080F31188BFF34F8FBFF36F8FFEE7606BE5
:105FC000A16B6163A063206A401C2062FFF788F820
:105FD000A06ADFF87880864209D3606B0068A0B1C0
:105FE000606BC068C5686868864211D2A06220688C
:105FF000C06A00EB800158F82100012800D9012770
:10600000E0690028C9D00127C7E74FF0FF30EDE76E
:10601000281DFFF79FF9A86A18B105F11800FFF7CE
:1060200099F9E86A2169884200D9206100EB800172
:1060300008EB8100291DFFF7DDF9E86A2168C96ACC
:106040008842CAD30127C8E7680000205003002017
:1060500070B504004FF0000133D01B4D2868844216
:1060600007D0502080F31188BFF34F8FBFF36F8F9D
:10607000FEE7206D38B1401E2065E36CE26A9A426B
:106080001FD040B11DE0502080F31188BFF34F8F27
:10609000BFF36F8FFEE7201DFFF75CF9E06CE06255
:1060A000C0F13800A061E06A2969884200D92861FE
:1060B000064900EB800001EB8000211DFFF79AF9F3
:1060C0000121084670BD0000680000205003002038
:1060D00070B5C068C46854B104F118000646FFF7F3
:1060E00039F9144D286B50B13146134815E0502052
:1060F00080F31188BFF34F8FBFF36F8FFEE7201D32
:10610000FFF728F9E06A2969884200D928610B491C
:1061100000EB800001EB8000211DFFF76BF9E06AC6
:106120002968C96A884202D90120E86170BD00204F
:1061300070BD000068000020D80700205003002038
:106140002DE9F0472C4D00242746286B38B1FFF786
:106150005DF9286B401E2863286B40B146E0502053
:1061600080F31188BFF34F8FBFF36F8FFEE7A968ED
:10617000224E0120D1B3A6F5916980463068E0B186
:10618000F068C46804F11800FFF7E4F8201DFFF779
:10619000E1F8E06A2969884200D9286100EB8001B2
:1061A00009EB8100211DFFF725F9E06A2968C96A1A
:1061B0008842E3D3C5F81C80E0E70CB1FEF790FFFE
:1061C000AC694CB14FEA0806FFF7DEFE00B1EE61A4
:1061D000641EF9D10020A861E86938B10849012797
:1061E00038070860BFF34F8FBFF36F8FFFF72EF9AB
:1061F0003846BDE8F087000068000020D80700207E
:1062000004ED00E010B586B0FEF7DCFC114C206810
:10621000B8B100200390049005AA04A903A8FFF7D1
:10622000B7F8DDE9032102208DE8070000230AA169
:106230000B48059AFFF768FE606010B106B00120B8
:1062400010BD502080F31188BFF34F8FBFF36F8FC5
:10625000FEE70000A4000020546D72205376630016
:10626000BD5100082DE9FF411E46134602000A9D5C
:106270004FF0000016D0144C2768002F0FD0CDE946
:1062800000130292062917DAFFF76AFE02284FF080
:1062900000030FD0002269462068FFF71FFC04B0FE
:1062A000BDE8F081502080F31188BFF34F8FBFF31A
:1062B0006F8FFEE72A46EEE70023324669463846EE
:1062C000FFF7BCFCEBE70000A4000020F46300082B
:1062D00000000000000000000000000000000000BE
:1062E0000002000018000000000000000000000094
:1062F000E86300080000000000000000000000004B
:106300000000000000020000180000000000000073
:1063100000000000146400080000000000000000FD
:10632000000000000000000000020000200000004B
:106330000000000000000000D06300080000000022
:10634000000000000000000000000000000000004D
:10635000DC63000800000000140100205000000071
:10636000F4000020200000001C6400080000000071
:1063700000000000000000000464000800000000AD
:10638000000000000000000000000000000000000D
:106390000102030406070809A0860100400D03005E
:1063A000801A060000350C0040420F0080841E0059
:1063B00000093D0000127A000024F40000366E014E
:1063C0000048E801006CDC02000000000102030448
:1063D0006D79517565756530310000006D795175C5
:1063E000657565303200000053656E6464617461E8
:1063F00000000000526561647072657373757265A8
:106400000000000064617461526561647953656DD8
:1064100000000000436F6D6D6F6E00006461746179
:106420004D75746578000000486400080000002085
:10643000F40000006C4200083C650008F4000020F5
:10644000F45400007C4200080000000000006400DA
:10645000010000000000000000000000000000003B
:10646000000000000000000000000000000000002C
:10647000000000000000000000000000000000001C
:1064800001000000100000000000000000000000FB
:1064900000000000000000000000000001000000FB
:1064A00000000000000000000000000000093D00A6
:1064B00000000000000000000000000000000000DC
:1064C00000000000000000000000000000000000CC
:1064D00000000000000000000000000000000000BC
:1064E00000000000000000000000000000000000AC
:1064F000000000000000000000000000000000009C
:10650000000000000000000000000000000000008B
:10651000000000000000000000000000000000007B
:106520000000000000000000AAAAAAAA00000000C3
:0C6530000000000000000000000000005F
:040000050800018D61
:00000001FF
